:020000020000FC
:1000000010E000E00A95F1F71A95E1F70BE501BB66
:1000100000E202BB00E008BB0FEF07BB50D0949A90
:100020004ED000E149D00A95E9F749D000E502BB7E
:1000300046D032D031D03CD02FD02ED035D034D095
:100040002BD02AD029D028D027D026D029D02CD0E8
:1000500027D02AD029D024D01FD01ED01DD01CD00C
:100060001BD022D021D018D017D01ED015D014D03C
:1000700013D012D011D010D017D016D00DD014D06C
:1000800013D00AD009D008D007D000E402BB17D0A3
:1000900000E002BBC09AFECF919890980DD00895D1
:1000A0009198909A09D00895919A909805D00895C2
:1000B000919A909A01D00895939A9398089500E1A7
:0600C0000A95F1F7089516
:00000001FF
